:100000000C9497030C94CF030C94CF030C94CF0360
:100010000C94CF030C94CF030C94CF030C94CF0318
:100020000C94CF030C94CF030C9448180C948A17AB
:100030000C94F5190C94CF030C94CF030C94CF03BC
:100040000C94CF030C94CF030C94CF030C94CF03E8
:100050000C94CF030C94B7190C94CF030C94CF03DA
:100060000C94CF030C94CF030C94CF030C94CF03C8
:100070000C94CF030C94CF030C94CF030C94CF03B8
:100080000C94CF030C94CF030C94CF030C94CF03A8
:100090000C94CF030C94CF030C94CF030C94CF0398
:1000A0000C94CF030C94CF030C94CF037A06EE0686
:1000B00082064C06500686065306890694065E069E
:1000C000E4066206980666069C06C6066A06A00650
:1000D000D0067006A606B00657068D065A0690068C
:1000E0007506AB06BC06DC06DE0648067E06F7068D
:1000F0001D0723071107170729072F073507510881
:10010000510884088408FE081F0A1F0A1F0A1C09D8
:100110009009A109A109BF0CC20CED0C060D0D0D33
:10012000180D1B0D1B0D1B0DE70DE70D500D520D8E
:10013000560D7B0D9C0D9F0DA20DC60DA215C91568
:100140007217C91572171516381672172D173D1725
:10015000FA1BF01B071C551C5B1C5B1C551C5B1C15
:100160005B1C281C5B1C321C3C1C5B1C5B1C5B1C52
:100170005B1C551C5B1C5B1C551C5B1C151C5B1C19
:100180005B1C571C571C571C571C571C571C571CD3
:10019000571C571C591C5B1CFA1BED1B5B1C5B1C82
:1001A0005B1C5B1C5B1C5B1C5B1C5B1C5B1C5B1C97
:1001B000591C5B1C5B1C551C5B1C4A1C4A1C4A1CC2
:1001C0004A1C4A1C4A1C4A1C4A1C4A1C591C000056
:1001D000000000000000000000000000000000001F
:1001E000000000000000000000000000000000000F
:1001F00000007E0F00D4FFFFFFC700000078000062
:100200000000000000002A2B280000000000000071
:1002100000000000000000000029000000002C1E6B
:100220003420212224342627252E362D3738271E28
:100230001F202122232425263333362E37381F044E
:1002400005060708090A0B0C0D0E0F1011121314E6
:1002500015161718191A1B1C1D2F3130232D3504A4
:1002600005060708090A0B0C0D0E0F1011121314C6
:1002700015161718191A1B1C1D2F3130354C050186
:100280000980A101850319012AB700150126B700CD
:10029000950175108100C0050C0901A101850419A3
:1002A000012AA002150126A002950175108100C047
:1002B00005010906A1018506050719E029E71500D2
:1002C00025019508750181020507190029EF150020
:1002D000250195F07501810205081901290595058B
:1002E00075019102950175039101C00660FF0961D6
:1002F000A1010962150026FF0095207508810209F9
:1003000063150026FF00952075089102C0050109BC
:1003100006A101050719E029E715002501950875D3
:100320000181029501750881010507190029FF1552
:100330000026FF00950675088100050819012905AA
:10034000950575019102950175039101C009025B44
:1003500000030100A0FA09040000010301010009E3
:100360002111010001224000070581030800010955
:1003700004010002030000000921110100012222F2
:10038000000705820320000107050303200001097F
:100390000402000103000000092111010001226D87
:1003A000000705840320000112010002000000087C
:1003B00000F178AD02000102000112034100640067
:1003C00065006C00680065006900640000001203AD
:1003D00066006C006F006F006F006B0061007900B9
:1003E00000000403090429003A003B003C003D00E2
:1003F0003E003F00400041004200430044004500F1
:1004000068004B0000000000000000000000000039
:1004100000000000000000000000000000000000DC
:10042000000035001E001F002000210022002300D4
:1004300024002500260027002D002E0031004C004E
:100440002B0014001A000800150017001C001800EB
:100450000C00120013002F0030002A004A00E000B8
:1004600004001600070009000A000B000D000E0032
:100470000F0033003400280000004D00E1001D0093
:100480001B0006001900050011001000360037009F
:100490003800E500000052004E00E0000000E200DD
:1004A00000002C00215200002C000000E60000009B
:1004B0000000500051004F00A600680069006A006B
:1004C0006B006C006D006E006F00700071007200B8
:1004D00073004600A90000000000000000000000BA
:1004E000000000000000000000000000000000000C
:1004F0000000000001003A003B003C003D003E00CF
:100500003F0040004100420043004400450001001C
:1005100049000100010001000100010001004A0042
:100520004E004B004D000100010001004C00057819
:10053000E300010001000100010001005000510032
:1005400052004F0001000100AE000000A8000100B1
:100550000100010001000100010001000100010093
:100560000100010001000000AE00AA00010000002F
:100570000100000001000100000001000000010076
:1005800000000000AC00AD00AB0001000100010064
:100590000100010001000100010001000100010053
:1005A0000100010001000100000000000000000047
:1005B000000000000000000000000000000000003B
:1005C0000000000000000100010001000100010026
:1005D0000100010001000100010001000100010013
:1005E0000100010001000100010001000100010003
:1005F00001000100010001000100010001000100F3
:1006000001000100010001000100010001000100E2
:1006100001000100010001000100010000000100D3
:1006200001000100010001000100010001000100C2
:1006300001000100010001000000010001000100B3
:1006400000000100000001000100000001000000A6
:100650000100000000000100010001000100010094
:100660000100010001000100010001000100010082
:100670000100010001000100010000000000000075
:10068000000000000000000000000000000000006A
:100690000000000000000000010001000100010056
:1006A0000100010001000100010001000100010042
:1006B0000100010001000100010001000100010032
:1006C0000100010001000100010001000100010022
:1006D0000100010001000100010001000100010012
:1006E0000100010001000100010001000100000003
:1006F00001000100010001000100010001000100F2
:1007000001000100010001000100000001000100E2
:1007100001000000010000000100010000000100D4
:100720000000010000000000010001000100112490
:100730001FBECFEFDAE0DEBFCDBF04B603FE18C0A8
:100740008091810290918202A0918302B0918402F3
:100750008730904BA740B04B59F410928102109211
:1007600082021092830210928402E0E0F8E309957D
:1007700011E0A0E0B1E0EEEAF1E402C005900D92D4
:10078000A436B107D9F722E0A4E6B1E001C01D927A
:10079000A138B207E1F70E94CC0A0C94D5200C9442
:1007A00000000E94501E2FEF84E39CE02150804007
:1007B0009040E1F700C000009CE088E10FB6F8949B
:1007C000A895809360000FBE90936000FFCFA7E1D3
:1007D000B0E0EDEEF3E00C94A0204B8B5C8B6D8BC6
:1007E0007E8B8F8B611110920E0286E09E01235F3B
:1007F0003F4FD901E82F1D92EA95E9F795E0FE01F8
:100800007396D90101900D929A95E1F79C894E89D2
:100810005F897B897D879E876F87598B488BF9011C
:10082000DE01179601900D928A95E1F7CE010796A9
:100830000E944E1281113EC086E0FE013796DE0115
:10084000119601900D928A95E1F7FF81E8856A85FE
:100850007B856115710531F0EF3F31F481E0FF3F99
:1008600019F403C081E001C080E080FD23C0209125
:10087000BB0130E0C9010196877099274091EC01D6
:1008800050E08417950779F1F983EA837D836C83BF
:1008900096E0929FD001939FB00D1124A454BE4FB7
:1008A000FE01319601900D929A95E1F78093BB017C
:1008B0000E94DB1116E08091EC019091BB01891739
:1008C000F9F0189FC001112484549E4F0E944E12CB
:1008D0008823B1F08091EC0190E001968770992710
:1008E0008093EC01E8CF0E94501E1092BB01109241
:1008F000EC01E5EBF1E086E0DF011D928A95E9F776
:100900006796E3E00C94BC20ADE0B0E0EAE8F4E0E8
:100910000C949120FC018081918123813481232BCF
:1009200031F09F3F31F491E08F3F19F403C091E023
:1009300001C090E090FDC1C57F0185E0DE01199600
:1009400001900D928A95E1F7F701228189859A85B8
:10095000222349F00E94551D182F682F89859A85FA
:100960000E94C51D03C00E94911D182F69857A85BC
:10097000812F0E942B0F8C01F7018281882309F4BB
:100980002CC19801225037472031310508F076C23A
:100990008FEF93E00E94E21F811128C102503EE6D2
:1009A000A32E33E0B32E002379F0A114F4E0BF06A8
:1009B00009F41CC1C5010E94E21F811101C0015050
:1009C0002FEFA21AB20AEFCFCE0101962C0188E0D8
:1009D000F20111928A95E9F72AE0322E85010F5F24
:1009E0001F4FC5010E94E21F89831A82882309F4E0
:1009F000FDC0813009F041C06501F2E0CF0ED11C8D
:100A0000C8010E94E21F8A83882309F4EFC09FEF88
:100A1000980F933060F423E0A20EB11CC6010E942F
:100A2000E21F8B83882309F4E1C01C8229C0843033
:100A300031F54E0133E0830E911C02E010E05601C7
:100A40008FEFA81AB80AC6010E94E21FF401819331
:100A50004F01882309F4CAC08C3741F4E2E0F0E08A
:100A6000EC0FFD1FE00FF11F10820AC00F5F1F4F38
:100A700065010730110519F7B9C0580101C05601C9
:100A80008201F8012081222309F4A8CF213009F046
:100A90004CC08181813049F46801F2E0CF0ED11C55
:100AA000F80182810E94C31F0AC0823051F468019C
:100AB000F2E0CF0ED11CF80182810E94DA1E86017D
:100AC00089C0833049F46801F2E0CF0ED11CF801EF
:100AD00082810E94811EF3CF843019F00F5F1F4F77
:100AE00079C0F80122810E5F1F4F80E090E030E076
:100AF000205331092A30310568F4389EA001399E0F
:100B0000500D1124C901840F951F0F5F1F4FF8016D
:100B10002081EDCF009709F45DC0EFE9FFE0319748
:100B2000F1F700C000000197F5CFE22FF0E0E250AE
:100B3000FE4F2490822F86958695869590E0FC0145
:100B4000E251FE4F64902770712C022E02C0759402
:100B500067940A94E2F7F1E06F227724FC01E252F5
:100B6000FE4F8490912C022E02C0959487940A9493
:100B7000E2F731E083229924FC01E253FE4FC49056
:100B8000D12C02C0D594C7942A95E2F781E0C822FF
:100B9000DD246114710419F081EE0E94DA1E8114C3
:100BA000910419F086EE0E94DA1E822D0E94C31F66
:100BB0008114910419F086EE0E94811E6114710463
:100BC00019F081EE0E94811EC114D10419F08CE24B
:100BD0000E94C31F0F5F1F4F54CF0115F7E71F0778
:100BE000B9F481E00E94FD1D0E94B3148091ED01D3
:100BF000877009F462C4F7018281882309F45DC417
:100C00008091160282FF59C482E00E94A71155C448
:100C1000013027E71207A9F482E0E4CF023038E779
:100C2000130709F43AC108F442C1043028E7120757
:100C300009F450C108F472C1053098E7190709F4A6
:100C40007DC1F801E851FC47E730F10508F4E5C043
:100C5000882309F4D4C110924B02C801905783979E
:100C600008F08CC184E090E00E94EA1F9093160285
:100C700080931502F801E150F047E232F10520F4CB
:100C8000EA5AFF4F0C946A20809115028160ACC033
:100C9000809116028860B4C0809115028260A4C061
:100CA0008091150220C08091150288609DC08091BE
:100CB00016021EC0809116028260A2C080911502A9
:100CC000806192C08091150280628EC08091150271
:100CD00080648AC00E94501E80911502806884C082
:100CE00080911502886084607FC0809116028260C6
:100CF000816086C0809115028E7F76C08091160239
:100D0000877F7EC0809115028D7F6EC08091150215
:100D100020C080911502877F67C0809116021EC097
:100D2000809116028D7F6CC0809115028F7E5CC011
:100D3000809115028F7D58C0809115028F7B54C021
:100D40000E94501E809115028F774EC0809115022F
:100D5000877F8B7F49C0809116028D7F8E7F50C028
:100D60008091150282FB222720F991E0922790FBC7
:100D700082F990FB83F938C080911602982F9095E4
:100D800091708E7F892B90FB81F93AC0809115027A
:100D900086FB222720F991E0922790FB86F924C058
:100DA0000E94501E8091150287FB222720F991E0B6
:100DB000922790FB87F918C061E001C060E08EE0E7
:100DC00090E00E94F01F1EC08091150284FB222734
:100DD00020F991E0922790FB84F906C080911502DA
:100DE000982F909590FB80F9809315020BC080910D
:100DF000160283FB222720F991E0922790FB83F9CA
:100E000080931602609115027091160284E090E0C2
:100E10000E940E200E94501EE9CEE858FF4F0C940D
:100E20006A2006E221EE41EE6AE17CE723C007E298
:100E300025EE45EE6BE17CE71DC006E221EE40EEBB
:100E400068E17CE717C007E225EE44EE69E17CE744
:100E500011C006E221EE42EE6CE17CE70BC007E236
:100E600025EE46EE6DE17CE705C008E221E045EEA7
:100E70006EE17CE7C7010E94D21AB8CE0115E7E700
:100E80001E0711F481E006C00130F7E71F0709F0E3
:100E9000C5CE82E00E940A1EA7CE8091940180FFF9
:100EA00003C00E94A70AA2CE0E94B40A9FCE0115D9
:100EB000E8E71E0711F483E006C00130F8E71F07DA
:100EC00009F0BFCE80E00E948D0A809194010E94BB
:100ED0004F1D8CCE20919401822F86958695869504
:100EE000482F50E04330510554F48F5F982F990FED
:100EF000990F990F822F8770892B8093940180918D
:100F000094018160809394010E944F1D809194010F
:100F10008695869586950E94AA1C68CE809194013C
:100F2000982F96959695969589F3915E990F990FBE
:100F3000990F8770892B8093940113C0909194012D
:100F4000892F8695869586958F5F8F71843090F472
:100F5000880F880F880F9770892B80939401809158
:100F60009401887F91E009F490E08091940190FBD6
:100F700080F9C8CF977090939401F1CF06312CE798
:100F8000120709F47AC203309CE7190721F140F4F3
:100F90000115FCE71F0789F001301C4711F134C02F
:100FA0000B353CE7130739F10C358CE71807D9F0FE
:100FB0000A351C4749F581E01FC00E94501EEFEF23
:100FC000F4E32CE0E150F0402040E1F700C00000E5
:100FD0000E9493190BCE6FEF7FEF80E090E00E94AC
:100FE0000E200E94D1038091160282FB882780F98F
:100FF00091E0892701C080E00E94C41105C006313C
:101000003CE7130709F449C2F7018281008111818D
:10101000882349F0C8010E94551DD82E682FC801A9
:101020000E94C51D04C0C8010E94911DD82EB801A0
:101030008D2D0E942B0F0E94390FB82E192F982E3C
:10104000F7010281A580A2949FE0A9228091ED0181
:101050008770B9F00023A9F0812F807F803421F0C0
:1010600080E28B0D883068F08091160282FF09C003
:1010700082E00E94A7118091ED018770DD24D39456
:101080008111D12CC12EC2948FE0C8228C2D90E00A
:101090008C30910508F0D3C1FC01E158FF4F0C944E
:1010A0006A20812F807F1F70882311F01295107F96
:1010B0000023B9F0112309F4B0C180E28B0D883010
:1010C00010F0911006C090910F02192B10930F028F
:1010D00005C090910E02192B10930E020E9452111E
:1010E0009CC18B2D0E94811E112309F4A8C180E2AE
:1010F0008B0D883088F1992079F1109590910E022E
:10110000192310930E022BC0812F807F1F70803215
:1011100011F01295107F8B2D992029F0F1E09F1688
:1011200009F441C04FC08091160282FD1BC000230C
:1011300069F0112339F090910F02192B10930F02CF
:101140000E94521180E00E94DA1E79C180E00E9464
:10115000811E112309F473C1812F0E944B110E943B
:1011600052116DC1002381F080911002AA2051F02C
:1011700021E0A21207C0182B181709F460C11093C0
:1011800010025DC1812B16C0A11003C00E94451141
:1011900031C031E0A31609F452C1812F0E94701EA4
:1011A0000E9445114CC1002341F085E08A1508F4E6
:1011B00046C1812F0E94771E42C194E09A1508F41F
:1011C0003EC118C0002349F0AA2099F3F701858198
:1011D00080FF23C18F708583ECCFAA2059F089331B
:1011E00009F02AC1FFEF27EE33E0F15020403040F4
:1011F000E1F720C1812F0E94701E21C1812F8695A9
:101200008695837019F0813061F019C1002321F0B7
:101210008B2D912F937002C080E090E00E94A01A65
:1012200014C1002321F08B2D912F937002C080E018
:1012300090E00E947B1A09C1812F8370A9F50111EA
:1012400002C14B2D429546954770440F440F8B2D9C
:101250008F7090E09C01042E01C0220F0A94EAF7DF
:10126000B4FE08C08FE090E001C0880F4A95EAF70D
:10127000809501C080E0169516951370123069F0C4
:1012800088F490911102113019F0822B892302C049
:10129000922B892B0E94161ED6C0822B9091110290
:1012A0008927F8CF822BF6CF002319F0812F817088
:1012B00001C08695882309F4C6C04B2D42954695FA
:1012C0004770440F440F8B2D8F7090E09C01042ECB
:1012D00001C0220F0A94EAF7B4FE08C08FE090E044
:1012E00001C0880F4A95EAF7809501C080E0169505
:1012F00016951370123059F078F49091460211301F
:1013000019F0822B892309C0922B892B06C0822BCE
:1013100090914602892701C0822B0E94FA1D93C03A
:101320001F70002339F0812F0E940A1E8B2D0E940E
:10133000771E89C08B2D0E94701E812F0E94FD1D7B
:1013400082C08B2D92EF991681F1991538F0E0EF5C
:101350009E1659F0F1EF9F1619F15BC023EF92161C
:1013600059F134EF9316C1F054C0002381F084E0AA
:101370008A1508F464C01F7181E090E0012E01C05D
:10138000880F0A94EAF790914602892720C095E0D9
:101390009A1508F454C0EFCF8091160282FD1AC04E
:1013A000002329F0812F8F7127C00023D9F3812FCB
:1013B0008F710E94FD1D43C0002341F01F7181E029
:1013C000012E01C0880F0A94EAF701C080E00E9454
:1013D000FA1D35C0002399F01F71812F0E940A1E4B
:1013E0008091160282FF07C0E8E01E9FC001112411
:1013F00083608093ED01812F0E940A1E20C081E04E
:101400000E94A711F1E0FA15D0F482E00E94A71122
:1014100016C0002321F0AA2029F28B2D94CEAA20F9
:1014200031F2893349F42FEF37EE83E02150304019
:101430008040E1F700C000008B2D0E94811E88EFE4
:101440008C0D843010F40E94C51ADD20B1F180911A
:10145000ED0180FD32C0F701128285958595859555
:101460000E940A1EC7010E9484048091ED018595A7
:10147000859585950E94FD1D20C080910F028A7A76
:1014800091E009F490E090936601811112C069E245
:1014900085E991E00E94461A09C080916601811198
:1014A0000AC069E285E991E00E941E1A0E94521169
:1014B0009DCB65E3EDCF65E3F5CF2D96E2E10C948E
:1014C000AD200E94D71081110AC00E94E3108091C4
:1014D000940184708961809394010E944F1D86E07D
:1014E00090E00E94E21F80939401282F2695269574
:1014F000269530E02430310524F087708861809390
:1015000094018091940180FF04C08695869586950C
:1015100001C080E00E94AA1C0895843008F083E096
:10152000909194019770282F220F220F220F922B57
:1015300090939401987F21E009F420E09091940128
:1015400020FB90F9909394010E94AA1C0895809129
:10155000940180FF08C08E7F809394010E944F1DEC
:1015600080E00E94AA1C08958091940180FD13C020
:10157000816080939401813019F489E08093940113
:10158000809194010E944F1D8091940186958695CB
:1015900086950E94AA1C0895ACE2B0E0E2EDFAE064
:1015A0000C94912085B7806885BF85B7806885BF1A
:1015B00084B7877F84BF0FB6F894A89580916000A8
:1015C000886180936000109260000FBE90E080E818
:1015D0000FB6F89480936100909361000FBE8FE086
:1015E0009EE090936501809364010E94CE170E9453
:1015F000ED178091E20084608093E20078948091FE
:101600003C028823A1F01091E9001F709091EC003A
:10161000892F817090FD80E8182B1092E90080914D
:10162000E80083FD0E94BF141F701093E90082E060
:1016300084BD93E095BD9AEF97BD80936E000E94A4
:10164000911C811102C00E94811C09E011E0D801A7
:101650008D918D018F3F11F00E94540EB1E0003149
:101660001B07A9F700E111E0F80181918F018F3F7D
:1016700011F00E94540EF1E00F311F07A9F78EE020
:10168000E6E8F1E0DF01282F1D922A95E9F7E7E669
:10169000F1E0DF011D928A95E9F70E94D7108111D0
:1016A00002C00E94E31082E090E00E94E21F80935B
:1016B000480284E090E00E94EA1F90931602809313
:1016C00015020E946B0EEFE3FCE93197F1F700C0C1
:1016D00000000E946B0E8091860180FF08C06FEFB2
:1016E0007FEF80E090E00E940E200E94931983E03B
:1016F00090E00E94E21F0E94161E3E9A469882E8E1
:101700008093900089E1809391008FEF9FEF9093F9
:101710009700809396000E94610A0E94610A80E00F
:1017200091E090934F0280934E028E010F5F1F4F06
:10173000CE010F969CA78BA780913C02853009F0C3
:101740004EC060E1E62E72E1F72E80913C028530BA
:1017500009F03FC080913C02843039F180E00E9462
:10176000AA1C10925202A8E1B0E0E0E40FB6F8948F
:10177000A895A09360000FBEE093600083B7817FBF
:10178000846083BF83B7816083BF7894889583B773
:101790008E7F83BF0FB6F894A89580916000886112
:1017A00080936000109260000FBE80913B028823FE
:1017B00009F4CBCF0E946B0EE6E8F1E081919191A4
:1017C000892B09F00DC284E991E08E179F07B1F7CC
:1017D000BCCF0E94501E0E94610A0E94C51A0E943E
:1017E0006B0E47E7C42E41E0D42E56E8E52E51E0BB
:1017F000F52ED701F601219131918D919D9182278E
:10180000932721E0E538F20719F0892BA1F322C0D4
:10181000892B01F50E94E9196C0180917501909165
:101820007601C816D90609F457C08FEF89A38AA399
:101830001BA20E94E9198160782F9DA38CA349A166
:101840005AA16BA18DA10E94E703D0927601C092AC
:10185000750142C036E8432E31E0532E312CD201BF
:101860008D909D902D01F60160807180682479240F
:101870006114710441F1212CAA24A394B12CC30159
:101880008A219B21892BB1F02EA23FA221E0C40125
:101890008A219B21892B09F420E028A70E94E919BD
:1018A0008160782F9AA789A74EA15FA168A58AA514
:1018B0000E94E7032394AA0CBB1CFFE02F12DFCF8A
:1018C000D6018D929C923394B2E0CB0ED11CE7E00E
:1018D0003E12C5CF0E94DD190E94C51A9091850164
:1018E000891721F0809385010E94DD1980913C02C7
:1018F000843009F021CF83E08093E9008091E800F3
:1019000082FF1ACF8091E80085FF23C00E941F1933
:1019100081111DC080E2C82ED12CCE0101965C0140
:1019200009C08091F100D5018D935D01B1E0CB1A22
:10193000D10869F08091E80085FDF3CF8091E8003F
:101940008B778093E8000E941F19882399F391E018
:1019500001C090E08091E8008B778093E8009923A4
:1019600009F4EACE2981822F90E0FC013197E3311E
:10197000F10508F02CC1E557FF4F0C946A201A823C
:101980008BE092C08A81823009F440C150F48130EA
:1019900009F01DC10E94DD199B838C837D836E83BA
:1019A00018C1833041F0843009F011C11B821C82C0
:1019B0001D821E820EC1FE013196D7018C911196B7
:1019C0009C91B2E0EB0EF11C9283838332968BA53F
:1019D0009CA58E179F0789F7FCC08A81823019F079
:1019E000853051F0F4C06B817C818D819E810E9495
:1019F00070200E945D1CEDC08091940180FF03C0A7
:101A00000E94A70AE6C00E94B40AE3C04C816B8121
:101A10008A810E94B31B9D8300C12D813E813227A4
:101A2000232732274C816B818A810E94571BD1C0AA
:101A30000E947E1BCEC08A81813009F0C8C0283048
:101A400099F0293041F18B81813009F0C2C08C813D
:101A5000A3E08A9FC00111246FEF70E00E94342040
:101A6000862F0E948D0AB5C08B81813029F082308B
:101A700009F0AFC01C82ADC0809194018695869517
:101A80008695BFEF8B9FC001112463E070E00E9438
:101A900034206C839EC0809194010E944F1D99C098
:101AA00080E14EC01A8282E98B8393C0EA80FB807A
:101AB000FE24EF24FE24AC80B12C6801C7018259BA
:101AC0009C4F9601201B310B2A153B0508F081C065
:101AD000E2E9EE16F10430F40E94E21FD6011496FA
:101AE0008C9302C0F6011482FFEFEF1AFF0A2FEF6A
:101AF000C21AD20AE3CFEA80FB80FE24EF24FE2440
:101B0000AC80B12C6801C70182599C4F9601201B03
:101B1000310B2A153B0508F05CC0A2E9EA16F10476
:101B200020F4F60164810E94F01FFFEFEF1AFF0A14
:101B30002FEFC21AD20AE7CF0E94471B4AC084E0A7
:101B40008A8347C0EA80FB80FE24EF24FE24AC8019
:101B5000B12C6801C70186969601201B310B2A150E
:101B60003B05B8F5A8E4EA16A3E0FA0628F40E94BB
:101B7000E21FF601848303C0D60114961C92BFEFC6
:101B8000EB1AFB0AEFEFCE1ADE0AE4CFEA80FB8005
:101B9000FE24EF24FE24AC80B12C6801C701869698
:101BA0009601201B310B2A153B0598F4F8E4EF163B
:101BB000F3E0FF0628F4D60114966C910E94F01F02
:101BC000BFEFEB1AFB0AEFEFCE1ADE0AE7CF8FEF7B
:101BD000898340E250E0B80182E00E945519ACCD03
:101BE000E9BCF9BC09B400FEFDCF8091D8008F7D1F
:101BF0008093D8008091E00082608093E000809123
:101C0000E00081FDFCCF0E94501E9FCD85E290E058
:101C10000E94E21F1B821C821D828E83DACF80E02D
:101C200008959091150292FF0DC0282F2871283039
:101C300019F4877F846006C0282F2471243011F4A2
:101C40008B7F886093FF0DC0282F2871283119F4ED
:101C5000877E846106C0282F2471243111F48B7E85
:101C600088612091160220FF0DC0382F387138305E
:101C700019F4877F816006C0382F3171313011F43B
:101C80008E7F886021FF0DC0282F2871283119F41C
:101C9000877E816106C0282F2171213111F48E7E4B
:101CA000886194FD877E0895F894E82FE295EF709F
:101CB000F0E031A1282F2F7081E090E001C0880F63
:101CC0002A95EAF7982F9095932391A392A1892BB7
:101CD00082A378940895AEE0B0E0E1E7FEE00C94D2
:101CE0009320AE014F5F5F4F7A018EE0FA011192AF
:101CF0008A95E9F709E011E06A0190E1492E91E047
:101D0000592E66246394712C3FE1832E31E0932E8B
:101D1000F80180818F3F09F446C0F894E82FE295DE
:101D2000EF70F0E021A18F70A30102C0440F551F96
:101D30008A95E2F7CA01922F982B91A392A18095E0
:101D4000892382A3789400C0E0E1F1E021E030E053
:101D5000A12CB12C41914F3F89F0A42FA295AF70D7
:101D6000B0E090968C9190E04F7002C09595879569
:101D70004A95E2F780FD02C0C90102C080E090E010
:101D8000A82AB92A220F331F8E169F0619F7F801C9
:101D900080818F3F11F00E94540EF0EAFA95F1F71E
:101DA000F601B182A0820F5F1F4FF2E0CF0ED11C6F
:101DB0004016510609F0ACCF4EE050E0B70187E67F
:101DC00091E00E94C820892B89F08EE0F701A7E6F8
:101DD000B1E001900D928A95E1F781E080931402C1
:101DE0000E94E919909313028093120280911402C9
:101DF000811102C080E02BC02091120230911302A9
:101E00004FB7F8948091530290915402A0915502DB
:101E1000B09156024FBF821B930B059758F34EE0CB
:101E200050E067E671E086E891E00E94C820892BC7
:101E300059F08EE0E7E6F1E0A6E8B1E001900D92FE
:101E40008A95E1F781E001C080E0109214022E969D
:101E5000E0E10C94AF20773048F46F3038F48430F0
:101E600028F4462F672F0E94B31B089580E090E06E
:101E70000895CF93DF938238910569F1B0F48133EF
:101E8000910509F477C048F48932910509F469C0D5
:101E90008A32910509F473C092C08533910509F423
:101EA0005BC089339105B9F08AC0833E910591F1F9
:101EB00038F4803E9105D1F0823E910531F17FC02A
:101EC000863E9105D9F1873E9105E9F1843E910561
:101ED00009F075C028C02091150220FD5BC021FDCE
:101EE00059C02091160223FD61C069C0809115027E
:101EF00080FD4AC08091160280FF4CC0809115027F
:101F000084FD50C183EE90E04FC18091150282FFA5
:101F10003EC0F4CF8091150282FD39C08091160237
:101F200080FD38C0EBCF8091160281FF39C08091CF
:101F3000150284FD37C187EE90E036C1809115020D
:101F400083FF2BC0F4CF8091150283FD26C08091C2
:101F5000160281FD25C0EBCF8091150285FD26C0BC
:101F600022C08091150285FD1EC08091160283FF5C
:101F70001DC00AC08091150286FD1BC01DC0809146
:101F8000150286FD19C015C089E390E00DC182EEEF
:101F900090E00AC180EE90E007C186EE90E004C1B7
:101FA00084EE90E001C185E390E0FEC089E290E01C
:101FB000FBC08AE290E0F8C081E390E0F5C0EC015C
:101FC000811530E5930708F053C0811560E496074A
:101FD00020F0CE019F70906AE7C0803E910588F5A1
:101FE0008D3C910518F0CE019065DEC0883A9105D0
:101FF000C0F4853A910550F08C2F855AC82FD0E057
:10200000C15EDE4F888190E09064CEC08130910542
:1020100009F4C5C008F4C6C0049708F4C3C0CE01D3
:10202000C3C0813C910508F0BDC08C2F885AC82FD1
:10203000D0E0CC0FDD1FCE5DDE4F888199819464A6
:10204000B3C08115904258F08D2F8F710E94110EF0
:10205000282F2F71CE0199279062922BA5C0C11510
:1020600081E0D807E0F6C83ED10508F09BC0D7CF85
:10207000C03692E5D90708F053C0C03422E5D20734
:10208000B8F08C2F8F718695869570E2879FA0019E
:1020900011248C2F837021E030E0B90102C0660F5B
:1020A000771F8A95E2F7CB019C68842B952B7CC027
:1020B000C03232E5D30740F08C2F8F7190E0982F1B
:1020C0008827816F906A70C0C11562E5D607B0F0AD
:1020D0008C2F8695869520E2829FA00111248C2F5B
:1020E000837021E030E0B90102C0660F771F8A9546
:1020F000E2F7CB01842B952B9D6856C08C2F8F71F6
:102100000E94110E95E0D695C7959A95E1F7CF708C
:10211000D0E0DC2FCC27D0699E01282BC90144C018
:10212000C03A72E5D70708F58C2F8F71C03892E559
:10213000D907A8F48695869570E2879F90011124AF
:102140008C2F837041E050E0BA0102C0660F771F08
:102150008A95E2F7CB019A68822B932B25C090E0F9
:10216000982F8827846F906A1FC0C03C22E5D20751
:1021700050F48C2F8F710E94110E8F7190E0982F68
:102180008827906211C0C03E32E5D30758F4CE01D3
:102190008F719927982F8827806F906A05C081E0FA
:1021A00090E002C080E090E0DF91CF91089580E060
:1021B00090E00E94EA1F873E9E4F19F40E94911CF6
:1021C000089580E0089567EE7EEF80E090E00E9441
:1021D0000E2060E082E090E00E94F01F60E083E06B
:1021E00090E00E94F01F1092110260E074E184E020
:1021F00090E00E940E2060E086E090E00E94F01FD8
:102200006FEF87E090E00E94F01F40E050E0BA01DD
:1022100088E090E00E94022060E08DE090E00E9463
:10222000F01F40E050E0BA0188E190E00E940220F7
:1022300060E087E190E00E94F01F40E050E0BA01CA
:102240008CE190E00E94022060E070E080E290E08B
:102250000E940E2040E050E0BA0188E190E00E9428
:10226000022080E00E94621C0E94811C40E050E03D
:10227000BA018FE090E00E94022040E050E0BA01F5
:1022800083E190E00E940220089580911002811164
:10229000109210020895809590910F0289238093E7
:1022A0000F02089590910F0280910E02982B909347
:1022B0009501809110028823D9F0892B8093950194
:1022C00080910801882331F08091150287FF02C0B8
:1022D0008EE101C086E0E7E9F1E090E0815028F06E
:1022E00021912223D9F39F5FF9CF91110E944511CB
:1022F00040E250E06EEE71E085E991E00E94C82076
:10230000892B21F180E2E5E9F1E0AEEEB1E0019048
:102310000D928A95E1F7E0914E02F0914F023097CD
:10232000A9F080910801882359F08091150287FF58
:1023300007C0809195018093960186E08093950176
:102340000280F381E02D85E991E0099508952091BF
:10235000ED01809582238093ED01982F977099F479
:1023600030E0482F082E000C550B2417350759F084
:102370009091160292FF07C08595859585950E94DC
:10238000FD1D1092ED0108959091160292FB2227F7
:1023900020F9281779F080FB92F99093160260914A
:1023A00015027091160284E090E00E940E2082E0F7
:1023B0000E94A71108958091EC019091BB018917AB
:1023C00019F08F5F8770FBCF08950F931F93CF9302
:1023D000DF938091BA0182958F7009F05AC0809185
:1023E000B701882309F455C08091EC011091BB011D
:1023F0006091B5017091B601C091B801D091B90159
:1024000091E06F3F09F090E0292F06E0811709F471
:1024100040C0209721F07F3F21F030E003C031E041
:1024200001C0322F90E030FD31C0089FF001099FBC
:10243000F00D1124DF01A454BE4F11963C91119769
:10244000371324C03C91361321C012963C91129749
:1024500031111CC013964D915C9114974C1B5D0B70
:10246000483C510598F48091BA018F708061809347
:10247000BA01EF53FE4F80818F708061808385EBBE
:1024800091E00E9484040E94DB1103C001968770D2
:10249000BDCFDF91CF911F910F910895A1E1B0E0E1
:1024A000E4E5F2E10C9498208C0185E0F801DE016E
:1024B0001D9601900D928A95E1F7F801E2809091C6
:1024C000B5016091B6014091B8015091B901411533
:1024D000510531F06F3F31F481E09F3F19F403C0A3
:1024E00081E001C080E0F82FF1709F2E80FD1BC1BC
:1024F000F80130812181C380D48085EBA82E81E052
:10250000B82EF090B701F601E41BF50BFF2009F49B
:10251000C7C08091BA01E83CF10508F092C0482F8D
:10252000407F09F051C0621311C093130FC0FE2CFD
:10253000E1100CC08F7080618093BA01C5010E94C8
:1025400084048091BA01F80185832AC1C114D104A1
:1025500031F02F3F31F481E03F3F19F403C081E0B7
:1025600001C080E080FD03C081E08E2502C080E0D4
:1025700090E0F82FF170FF2E80FF1CC08091EC01DD
:102580004091BB0156E0841709F4E8C090E0589FE1
:10259000F001599FF00D1124E454FE4F6181261380
:1025A00006C06081631303C06281E61203C0019616
:1025B0008770E9CFFE2CEE2009F4F2C08091BA01B9
:1025C00081608093BA0149C0621306C0931304C0AE
:1025D000E11002C0F80186C0C8010E94191E8823BC
:1025E00051F1EE2041F12091BA01822F82958F7036
:1025F00090E0029774F08091B5019091B6019887B0
:102600008F831986DB86CA862C87CE0107960E94A7
:10261000840486E0F801A5EBB1E001900D928A9563
:10262000E1F70E94E5110AC06217C9F0C8010E94D3
:10263000191E81111EC0C8010E948404FF24F39456
:10264000AFC0482F407F81F785EB91E00E94840462
:1026500086E0F50111928A95E9F7F12CA1C0931358
:10266000E5CFE110E3CFF8018583C8010E9484041F
:1026700054C0EE2001F32091BA01822F82958F7011
:1026800090E0029734F28091B5019091B6019A835F
:1026900089831B82DD82CC822E83CE010196B7CF47
:1026A000E83CF105D0F5FE2CEE2029F2621327C09C
:1026B000931325C02091BA0120FD18C0822F829566
:1026C0008F70482F50E04115510581F0F8012583A6
:1026D0004F30510541F08F5F982F9295907F822F58
:1026E0008F70892B8583C8010E94840486E0F801DD
:1026F000A5EBB1E001900D928A95E1F751C0C801B8
:102700000E94191E811185CF8091BA01816080934A
:10271000BA01C8010E94840443C086E0F501119209
:102720008A95E9F73DC0EE2009F485CFC8010E94E3
:10273000191EF82E882309F47ECF86E0F801A5EB58
:10274000B1E001900D928A95E1F78091B5019091E9
:10275000B6010E94841D0E94E51122C03D872E878C
:102760008D859E850E94841D292F22952F702230F1
:1027700028F49F7039F0811105C00BC0243028F473
:102780009F7049F4805E883020F0C8010E94840464
:102790009F2CF92C05C0F8019581907F99F7F9CF0E
:1027A0008F2D6196EBE00C94B42080913E0287FF60
:1027B00011C08091E80082FD05C080913C0281112A
:1027C000F8CF11C08091E8008B770BC080913C025C
:1027D000882349F08091E80080FFF8CF8091E800DD
:1027E0008E778093E8000895982F973068F590933E
:1027F000E900981739F07091EC002091ED005091AC
:10280000F00003C0242F762F50E021FD02C09F5F0F
:10281000ECCF3091EB003E7F3093EB003091ED0038
:102820003D7F3093ED003091EB0031603093EB0051
:102830007093EC002093ED005093F0002091EE0097
:1028400027FDE5CF80E008958F708093E90081E057
:10285000089520914402309145022617370748F029
:102860006115710539F42091E8002E772093E80076
:1028700001C0B901FC0120E06115710579F1809179
:102880003C028823F1F18530F1F18091E80083FD6D
:102890003CC08091E80082FD2EC08091E80080FF5E
:1028A000EBCF2091F3008091F20090E0922B611524
:1028B000710551F08830910538F421912093F10091
:1028C000615071090196F3CF21E0089709F020E0EB
:1028D0008091E8008E778093E800CECF2111CFCF92
:1028E0000AC080913C02882361F0853061F08091BC
:1028F000E80083FD0AC08091E80082FFF2CF80E00B
:10290000089582E0089583E0089581E00895089590
:1029100043E050E0BC0184E00E9455190895CF9334
:10292000DF93EC0180910801811105C048E050E07F
:10293000BE0181E00BC08091150287FF03C040E219
:1029400084E002C048E081E050E0BE010E945519D9
:1029500080E2FE01AAE1B2E001900D928A95E1F7D2
:10296000DF91CF91089580914602982F967096300E
:1029700011F4886001C0877F0E94FA1D0895AAE2C1
:10298000B0E0E5ECF4E10C94A020EEE3F2E086E4A4
:1029900092E02091F10021938E179F07D1F780914B
:1029A0003F02833009F463C030F4813071F082302B
:1029B00009F49DC0B4C08A3009F489C08B3009F491
:1029C0006EC0893009F0ABC020C080913E02813AD0
:1029D00009F0A5C08091E800877F8093E80080918E
:1029E000420290914302892B21F460E28AE192E055
:1029F00003C060E080E090E070E00E9429148091C4
:102A0000E8008B778093E8008AC080913E02813293
:102A100009F085C08091420290914302009719F01D
:102A2000029709F07CC08091E800877F8093E800DE
:102A30008091E80082FD05C080913C028111F8CFB1
:102A40006EC02091F3008091F20090E0922B0297EB
:102A500031F48091F100813011F0863021F48091C1
:102A6000F100809319028091E8008B7754C0809127
:102A70003E02813A09F053C0809142029091430294
:102A8000892B09F04CC08091E800877F8093E80093
:102A90008091E80080FFFCCF8091080137C08091D1
:102AA0003E028132E1F58091420290914302892BEE
:102AB000B1F58091E800877F8093E8000E94D513EC
:102AC00080914002809308010E94501E28C080918E
:102AD0003E02813221F58091E800877F8093E800F3
:102AE0000E94D513809141028093180218C08091F2
:102AF0003E02813AA1F48091E800877F8093E8004C
:102B00008091E80080FFFCCF809118028093F10053
:102B10008091E8008E778093E8000E94D513809121
:102B2000E80083FFDFC180913E0290913F02492F70
:102B300050E04A30510508F0D5C1FA01E256FF4F86
:102B40000C946A20803821F0823809F0CBC108C08B
:102B500080913A0290913B02992389F082600FC0E4
:102B6000809142028F70873008F0BCC18093E900E9
:102B70008091EB0085FB882780F91092E900909105
:102B8000E800977F9093E8008093F1001092F100A5
:102B900070C1282F2D7F09F0A5C1882319F082303C
:102BA00061F0A0C180914002813009F09BC1933057
:102BB00009F080E080933B022EC080914002811199
:102BC0002AC0809142028F702FEF280F263008F024
:102BD00089C18093E9002091EB0020FF1CC0933055
:102BE00021F48091EB00806214C09091EB00906121
:102BF0009093EB0021E030E0A90102C0440F551F83
:102C00008A95E2F74093EA001092EA008091EB0087
:102C100088608093EB001092E9008091E800877F44
:102C20008093E8000E94D5135DC181115BC11091B2
:102C300040021F778091E3008078812B8093E3002E
:102C40008091E800877F8093E8000E94D5138091EF
:102C5000E80080FFFCCF8091E30080688093E30070
:102C6000111102C082E001C083E080933C023AC1AE
:102C70008058823008F036C12091400230914102E4
:102C80002C3D53E0350779F583E08A838AE2898316
:102C90004FB7F894DE01139620E03EE051E2E32FB7
:102CA000F0E050935700E49120FF03C0E295EF70ED
:102CB0003F5FEF708E2F90E0EA3010F0C79601C0B2
:102CC000C0968D939D932F5F243149F74FBF80911C
:102CD000E800877F8093E8006AE270E0CE01019609
:102CE0000E942914B4C08091420290914302432F64
:102CF000552743305105A9F068F44130510509F4D6
:102D000000C14230510509F0EDC08BE590E0EDE4E3
:102D1000F3E04BC04132510529F14232510589F1AE
:102D2000E1C0C901992781309105A1F058F00297BF
:102D300009F0D8C0EAEBF3E0E4918E2F90E0EAEBE3
:102D4000F3E030C0E2EEF3E0E4918E2F90E0E2EEAB
:102D5000F3E028C0EEECF3E0E4918E2F90E0EEEC8F
:102D6000F3E020C08330910508F0BCC0880F991FA4
:102D7000FC01E35AFE4F0190F081E02D89E090E0E4
:102D800014C08330910508F0ADC0FC01EE0FFF1FA9
:102D9000E95AFE4F0190F081E02DDC01AC5ABE4FA4
:102DA0008C9190E0009709F49DC02091E800277F66
:102DB0002093E800209144023091450228173907FA
:102DC00008F4C90140E0009789F120913C022223D8
:102DD00009F43DC02530D9F12091E80023FD37C02A
:102DE0002091E80022FD2FC02091E80020FFEBCFCA
:102DF0004091F3002091F20030E0342B009759F01D
:102E00002830310540F444914093F1003196019708
:102E10002F5F3F4FF3CF41E02830310509F040E00C
:102E20002091E8002E772093E800CDCF4111CDCF3F
:102E30000AC080913C02882351F0853041F0809196
:102E4000E80083FD04C08091E80082FFF2CF80910A
:102E5000E8008B778093E80045C0803809F042C0D5
:102E60008091E800877F8093E80080913D02809305
:102E7000F1008091E8008E77D3CE811133C080912C
:102E80004002909141029927029764F58091E800F1
:102E9000877F8093E8001091400210933D020E94CA
:102EA000D513111106C08091E30087FD02C081E0B7
:102EB00001C084E080933C0242E061EC81E00E942A
:102EC000F41342E261EC84E00E94F41342E261EC0C
:102ED00082E00E94F41342E260EC83E00E94F4136B
:102EE00080913C028091E80083FF10C08091E8004F
:102EF000877F8093E8008091EB0080628093EB00F5
:102F000005C082E190E0E8EAF3E04FCFAA96E3E063
:102F10000C94BC201F920F920FB60F9211242F9386
:102F20003F934F935F936F937F938F939F93AF9351
:102F3000BF93CF93DF93EF93FF93C091E900CF70DE
:102F40008091EC00D82FD17080FDD0E81092E9007C
:102F50008091F000877F8093F00078940E94BF14E6
:102F60001092E9008091F00088608093F000CD2BF2
:102F7000CF70C093E900FF91EF91DF91CF91BF91A6
:102F8000AF919F918F917F916F915F914F913F9101
:102F90002F910F900FBE0F901F901895E8EDF0E065
:102FA00080818E7F80831092E2001092DA0010926E
:102FB000E100A0EEB0E08C9181608C9380818F77EE
:102FC000808319BCA7EDB0E08C918E7F8C938081BB
:102FD0008F7E8083109217020895A0E0B0E0E3EFA7
:102FE000F7E10C949B20C8EDD0E088818F7E888328
:102FF000E7EDF0E080818160808384E082BF81E042
:103000008093170288818E7F888302EE10E0F8019A
:1030100010821092DA0081EEC82ED12CF6011082B7
:1030200088818F77888388818068888388818F7D75
:10303000888319BC10923C0210923D0210923B0210
:1030400010923A0290EEE92EF12CF70180818B7FED
:10305000808388818160888342E060E080E00E9414
:10306000F413F60180818E7F8083F8018081816076
:103070008083808188608083F70180818E7F808358
:10308000888180618883CDB7DEB7E8E00C94B720F3
:103090001F920F920FB60F9211242F933F934F93CD
:1030A0005F936F937F938F939F93AF93BF93EF93B0
:1030B000FF938091E10082FF09C08091E20082FFCE
:1030C00005C08091E1008B7F8093E1008091DA0060
:1030D00080FF2AC08091D80080FF26C08091DA004E
:1030E0008E7F8093DA008091D90080FF18C080E144
:1030F00089BD82E189BD09B400FEFDCF81E08093E6
:103100003C028091170281110FC00E94CE170E94CD
:10311000ED178091E20084608093E20005C019BC45
:1031200010923C02109217028091E10080FF17C0BC
:103130008091E20080FF13C08091E2008E7F809337
:10314000E2008091E20080618093E2008091D800EB
:1031500080628093D80019BC85E080933C02809106
:10316000E10084FF30C08091E20084FF2CC080E148
:1031700089BD82E189BD09B400FEFDCF8091D800F0
:103180008F7D8093D8008091E1008F7E8093E10055
:103190008091E2008F7E8093E2008091E200816066
:1031A0008093E20080913D02882311F084E007C003
:1031B0008091E30087FD02C081E001C083E080933D
:1031C0003C0280913C028091E10083FF27C0809106
:1031D000E20083FF23C08091E100877F8093E100BC
:1031E00082E080933C0210923D028091E1008E7F4C
:1031F0008093E1008091E2008E7F8093E2008091D5
:10320000E20080618093E20042E060E080E00E94A2
:10321000F4138091F00088608093F000FF91EF91AB
:10322000BF91AF919F918F917F916F915F914F91DE
:103230003F912F910F900FBE0F901F9018952091E6
:10324000E4003091E50095E64091EC00842F817018
:1032500040FF23C08091E80080FD1DC080913C02AA
:10326000882399F0853099F08091EB0085FD11C09D
:103270004091E4005091E5002417350729F391505F
:1032800011F09A01E1CF84E0089582E0089583E08F
:10329000089581E0089580E008954091E80042FF9C
:1032A000DDCF08958091190208950F931F93CF9356
:1032B000DF938B01EA0190913C02943079F58F7095
:1032C0008093E9008FEF9091E800815095FD06C052
:1032D00095ED9A95F1F700008111F5CF8091E80006
:1032E00085FF1CC00E941F19882361F08091E800AF
:1032F0008E778093E80012C0F80181918F0180934E
:10330000F1002197209791F38091E80085FDF4CF9B
:103310008091E8008E778093E800E4CFDF91CF9131
:103320001F910F91089581E08093E00080E28093E7
:10333000D8001092C9008FE19EE40197F1F700C018
:10334000000087E090EBDC01809381029093820281
:10335000A0938302B09384029CE088E10FB6F894B6
:10336000A895809360000FBE90936000FFCF789483
:103370001F920F920FB60F9211248F939F93AF93CA
:10338000BF938091530290915402A0915502B09145
:1033900056020196A11DB11D8093530290935402D1
:1033A000A0935502B0935602BF91AF919F918F9118
:1033B0000F900FBE0F901F9018952FB7F894609143
:1033C00053027091540280915502909156022FBF82
:1033D00008952FB7F8948091530290915402A091D0
:1033E0005502B09156022FBF08951F920F920FB64B
:1033F0000F9211248F939F93AF93BF9380915202AA
:10340000811113C08091530290915402A0915502F2
:10341000B09156024196A11DB11D80935302909325
:103420005402A0935502B0935602BF91AF919F9161
:103430008F910F900FBE0F901F901895209108014B
:103440002223C9F02091150227FF15C0262F2695AB
:10345000269526952E31C8F4FC01E20FF11D677008
:1034600081E090E001C0880F6A95EAF7809592812B
:10347000892382830895FC0106962281621301C08C
:1034800012823196E817F907C1F7089520910801D3
:103490002223C1F02091150227FF14C0262F269564
:1034A000269526952E3130F5FC01E20FF11D67704F
:1034B00081E090E001C0880F6A95EAF79281892B3C
:1034C00082830895FC0132962FEF30E0419164171A
:1034D00089F02F3F19F4411101C0232F3F5F36308F
:1034E000A9F72F3F39F0FC01E20FF11D27FDFA95F6
:1034F000628308950895A3E0B0E0E1E8FAE10C9456
:10350000A120209150023091510228173907A1F0D3
:103510009093510280935002E0914E02F0914F023D
:10352000309751F024E029839B838A830680F781BA
:10353000E02DCE01019609952396E2E00C94BD2082
:10354000A3E0B0E0E6EAFAE10C94A12020914C025D
:1035500030914D0228173907A1F090934D028093C6
:103560004C02E0914E02F0914F02309751F023E06F
:1035700029839B838A830680F781E02DCE01019603
:1035800009952396E2E00C94BD20E0914E02F09163
:103590004F02309729F00190F081E02D09950895B0
:1035A00080E008950F931F93CF93DF93C42F122FC2
:1035B000FC0182818823B1F040934B020E94E919FB
:1035C00090934A028093490280E28C0F883008F081
:1035D00059C0C77081E001C0880FCA95EAF70E9400
:1035E000771E50C080914B0248133CC02091490285
:1035F00030914A024FB7F89480915302909154024F
:10360000A0915502B09156024FBF821B930B883C8C
:10361000910540F5D0E2D10FC117B9F080E28C0FCF
:10362000883040F4C77081E001C0880FCA95EAF77E
:103630000E94701ED83018F581E0912F977001C05C
:10364000880F9A95EAF70E94771E802F0E94C31F69
:10365000D830C0F4212F277081E001C0880F2A954F
:10366000EAF70AC080E28C0F883060F4C77081E00E
:1036700001C0880FCA95EAF70E94701E03C0802F10
:103680000E94C31FDF91CF911F910F910895CF9397
:10369000DF93CEE6D3E060E0CE010E94F01F2196DA
:1036A000C11584E0D807B9F7DF91CF9108951F9332
:1036B000CF93DF93962F8430E8F46730D8F44F30FF
:1036C000C8F4632F122FC42FD0E0CC0FDD1F2EE1E2
:1036D000929FC00DD11D112492ED899FC00DD11D67
:1036E0001124CE0186960E94F01F612FCE0187968D
:1036F0000E94F01FDF91CF911F910895A0E0B0E0EC
:10370000E4E8FBE10C949920A12CE12CF12CB12CE4
:1037100000E010E0C0E0D0E06701C00ED11EFE0165
:10372000EE0FFF1FEC0DFD1DEA51FC4F259134916A
:103730004C2F6B2D8A2D0E94571B2196CF30D1051F
:1037400071F7025E1F4FB39487E0B812E3CF82EDAA
:10375000E80EF11CA39484E0A812D9CFCDB7DEB750
:10376000EAE00C94B5200F931F93CF93DF9384303E
:1037700008F56730F8F44F30E8F4C42FD0E0CC0FF0
:10378000DD1F2EE1629FC00DD11D112432ED839FFC
:10379000C00DD11D1124CE0186960E94E21F90E03B
:1037A000182F0027CE0187960E94E21F9801282B30
:1037B000C90102C080E090E0DF91CF911F910F918D
:1037C0000895482F50E0FA013597EF33F10508F0DE
:1037D00072C0E855FF4F0C946A200E94E31065C048
:1037E00080914802817F8E7F8093480281E08093A0
:1037F000470208950E94501E2FEF84E39CE0215061
:1038000080409040E1F700C000000E949319809131
:103810004802982F9095917090FB80F98093480210
:10382000911143C0897F877F10C08091480281FB3E
:10383000222720F991E0922790FB81F9809348029A
:10384000992399F1809148028160809348022DC0AC
:103850008091480282FB222720F991E0922790FB79
:1038600082F9ECCF8091480283FB222720F991E076
:10387000922790FB83F9E2CF0E94501E809115029F
:1038800087FB222720F991E0922790FB87F980930C
:1038900015020BC0895391E001C0990F8A95EAF790
:1038A000892F0E94161E0E94501E81E008958D519E
:1038B000F2CF81E0F6CF80E0089585E290E00E94AB
:1038C000F01F0895CF93C82F811102C06FEF01C080
:1038D00062E282E290E00E94F01FC11102C06FEF2D
:1038E00001C062E183E290E00E94F01FC11102C0BA
:1038F0006FEF01C068E084E290E00E94F01FCF917A
:10390000089580E00E94621C60E070E0CB010E949C
:103910005D1C0E947E1B0E94471B81E00E94621C6E
:10392000089582E290E00E94E21F823281F483E2F5
:1039300090E00E94E21F823151F484E290E00E9404
:10394000E21F91E0883009F090E0892F01C080E00B
:1039500081700895A0E0B0E0E0EBFCE10C949720CA
:10396000843048F4811108C0909190009F77909323
:103970009000469806C083E09091900090689093E4
:103980009000A0919600B0919700282F30E00E94FF
:10399000772023E030E040E050E00E9448200027FC
:1039A000122F232F342F012F122F232F33278091F3
:1039B0009600909197006CE070E00E9434206017B0
:1039C000710730F0C80169E070E00E9434205EC0E9
:1039D0008091960090919700E0909600F09097006B
:1039E000E0919600F0919700C6E0D0E0BE010E9401
:1039F0003420060F171F211D311D4801590185E094
:103A0000880C991CAA1CBB1C8A95D1F7C701BE0162
:103A10000E9434206F01E12CF12CA7019601260FA2
:103A2000371F411D511DC501B4010E944820690185
:103A30007A01E0919600F0919700CA01B9010E94C5
:103A400024209B01AC01DF010E9486209B01AC0178
:103A5000C701B6010E942420DC01CB012FE0B695FE
:103A6000A795979587952A95D1F700919600109183
:103A7000970020E030E0081719072A073B0728F4D1
:103A80006091960070919700CB01BC0170939900F2
:103A900060939800CDB7DEB7ECE00C94B320682FAC
:103AA00086E090E00E94F01F0895CF92DF92FF928F
:103AB0000F931F93CF93DF936C0100914602809187
:103AC0001102082BC7E0D0E010E0C8010C2E02C0A4
:103AD000959587950A94E2F780FD04C02197A8F791
:103AE000F12C09C0FC2EB6018C2F0E942B0F0E94D6
:103AF000390F019799F38F2DDF91CF911F910F917E
:103B0000FF90DF90CF900895CF93DF93EC010E9458
:103B1000551DBE010E942B0F0E94390FDF91CF91DE
:103B20000895292F973078F58F3068F590E03FE0C1
:103B3000239F800D911D1124682F677023E09695B7
:103B400087952A95E1F7FC01EE0FFF1FE80FF91F9B
:103B5000E95AFD4F40E050E080E0219130E0062E30
:103B600002C0369527950A94E2F721703327042E78
:103B700001C0220F0A94EAF7822B4F5F5F4F433058
:103B8000510559F7089580E00895292F973088F559
:103B90008F3078F590E03FE0239F800D911D112438
:103BA000282F277051E001C0550F2A95EAF723E02E
:103BB000969587952A95E1F7FC01EE0FFF1FE80F18
:103BC000F91FE95AFD4F20E030E070E04081CB0161
:103BD000022E02C0969587950A94E2F7817081952E
:103BE00084278523842781932F5F3F4F233031051E
:103BF00069F7089580934602089521E030E001C0FE
:103C0000220F8A95EAF720958091460282230E942E
:103C1000FA1D089521E030E001C0220F8A95EAF7ED
:103C200080914602822B0E94FA1D08958093110212
:103C30000895CF93FC018081918123813481232BCE
:103C400031F09F3F31F491E08F3F19F403C091E0D0
:103C500001C090E0C92FC17090FD1CC0808191818E
:103C60000E94841D92959F70963079F010F49250C6
:103C700001C09A50923088F4803F71F018F4883E69
:103C800060F40AC0843F49F407C0883E28F0813FB1
:103C900021F402C0C0E001C0C1E08C2FCF91089593
:103CA00010920F0280910801882331F08091150253
:103CB00087FF02C08EE101C086E0E7E9F1E0DF01A5
:103CC0001D928A95E9F780E090E00E94A01A80E0BA
:103CD00090E00E947B1A10920E020E9452110895E9
:103CE000882321F00E944B110E94521108958823CD
:103CF00039F090910F02892B80930F020E9452118C
:103D00000895882309F455C0682F823869F40E9409
:103D1000C51A81FF4EC069E385E991E00E94461A09
:103D20000E94521169E30EC0833899F40E94C51AAB
:103D300080FF3FC063E585E991E00E94461A0E943A
:103D4000521163E585E991E00E941E1A0E9452110A
:103D50000895843869F40E94C51A82FF2AC067E476
:103D600085E991E00E94461A0E94521167E4EACF69
:103D70008CEF860F813A30F380E2860F883048F46A
:103D8000677081E001C0880F6A95EAF70E944B11C5
:103D9000DDCF8BE5860F833028F480E090E00E9431
:103DA000A01A0895685A693120F480E090E00E94DA
:103DB0007B1A0895CF93882309F4E3C0C82F823873
:103DC000B1F40E94C51A81FDDCC069E385E991E088
:103DD0000E94461A0E9452112FEF87EE93E0215065
:103DE00080409040E1F700C0000069E317C08338CD
:103DF000E1F40E94C51A80FDC4C063E585E991E045
:103E00000E94461A0E9452112FEF81EE94E0215039
:103E100080409040E1F700C0000063E585E991E053
:103E20000E941E1A0E945211ACC08438B1F40E9444
:103E3000C51A82FDA6C067E485E991E00E94461A92
:103E40000E9452112FEF81EE94E02150804090406B
:103E5000E1F700C0000067E4E1CF8CEF8C0F813AFE
:103E600040F580914702882319F0813051F01EC03F
:103E700080910F02823209F04CC08C2F0E94E11B0E
